:100000000C9465020C94A9020C94A9020C94A90208
:100010000C94A9020C94A9020C94A9020C94A902B4
:100020000C94A9020C94A9020C94430D0C94150E87
:100030000C942B1C0C94A9020C94A9020C94A902F8
:100040000C94A9020C94A9020C94A9020C94A90284
:100050000C94A9020C94981C0C94A9020C94A9026B
:100060000C94A9020C94A9020C94A9020C94A90264
:100070000C94A9020C94A9020C94A9020C94A90254
:100080000C94A9020C94A9020C94A9020C94A90244
:100090000C94A9020C94A9020C94A9020C94A90234
:1000A0000C94A9020C94A9020C94A90235001E001C
:1000B0001F0020002100220023002400250026002C
:1000C00027002A002B0014001A0008001500170052
:1000D0001C0018000C00120013002A002900040064
:1000E0001600070009000A000B000D000E000F00AB
:1000F00033003400E1001D001B000600190005005C
:100100001100100036003700380028000030E000F1
:10011000E200E30003522C002C0004525000510076
:1001200052004F0035001E001F0020002100220059
:10013000230024002500260027002A002B0014009D
:100140001A00090013000A000D000F0018001C001F
:1001500033002A00290004001500160017000700CC
:100160000B00110008000C0012003400E1001D001B
:100170001B000600190005000E00100036003700B5
:10018000380028000030E000E200E30003522C00B9
:100190002C0004525000510052004F0035001E0048
:1001A0001F0020002100220023002400250026003B
:1001B00027002A002B0034003600370013001C00F3
:1001C00009000A00060015000F002A00290004009B
:1001D0001200080018000C0007000B0017001100A7
:1001E00016003800E100330014000D000E001B0063
:1001F000050010001A0019001D0028000030E00062
:10020000E200E30003522C002C0004525000510085
:1002100052004F0035001E001F0020002100220068
:10022000230024002500260027002A0035021E0294
:100230001F0220022102220223022402250226029A
:1002400027022A0001003A003B003C003D003E002E
:100250003F002D022E022F02300231020100400029
:100260004100420043004400450000530153025343
:100270000050010001000100010001000100010027
:1002800001000100AB00AA00A900AE0035001E006D
:100290001F0020002100220023002400250026004A
:1002A00027002A0035001E001F0020002100220028
:1002B000230024002500260027002A0001003A0020
:1002C0003B003C003D003E003F002D002E002F0073
:1002D0003000310001004000410042004300440072
:1002E000450000530153025300500100010001007A
:1002F000010001000100010001000100AB00AA00A3
:10030000A900AE002A0354006800650020005000D8
:10031000720065006F006E006900630020004B00F2
:100320006500790062006F006100720064000000E7
:100330002C034F007200740068006F006C006900AD
:100340006E0065006100720020004B0065007900BE
:1003500062006F006100720064007300000004031B
:10036000090409027400040100A0FA090400000154
:1003700003010100092111010001223F000705814D
:100380000308000A09040100010301020009211108
:10039000010001224D000705820308000A0904023A
:1003A00000010300000009211101000122360007AD
:1003B00005830308000A0904030002030000000982
:1003C00021110100012220000705840320000107FC
:1003D0000504032000011201100100000008EDFED9
:1003E00061600100010200010631FF0974A10109E9
:1003F00075150025FF9520750881020976150025E1
:10040000FF952075089102C005010980A1018502B0
:1004100016010026B7001A01002AB70075109501D1
:100420008100C0050C0901A1018503160100269C6D
:10043000021A01002A9C02751095018100C0050175
:100440000902A1010901A1000509190129051500E9
:10045000250195057501810295017503810105014D
:10046000093009311581257F950275088106093803
:100470001581257F950175088106050C0A3802153E
:1004800081257F950175088106C0C005010906A177
:1004900001050719E029E715002501950875018177
:1004A0000295017508810105081901290595057551
:1004B0000191029501750391010507190029FF15A6
:1004C0000025FF950675088100C011241FBECFEFDF
:1004D000DAE0DEBFCDBF04B603FE24C08091F10197
:1004E0009091F201A091F301B091F4018730904B0B
:1004F000A740B04BB9F41092F1011092F2011092A2
:10050000F3011092F40114BE84B7877F84BF88E1A1
:100510000FB6F89480936000109260000FBEE0E088
:10052000F8E3099511E0A0E0B1E0E0EEF9E402C0E3
:1005300005900D92A435B107D9F711E0A4E5B1E01B
:1005400001C01D92A13FB107E1F70E94720A0C940D
:10055000EE240C94000061110DC0FC0182818823FF
:1005600031F085EE0E9426110E94272303C085EEFC
:100570000E94EE1180E090E00895089508950E9491
:10058000D1026E9A769A8DEB92E0892B11F00C9441
:10059000BD0208958EEB92E0892B11F00C94BE02FF
:1005A0000895279A2F988FEF9FEF9093870080935D
:1005B00086008AE08093800089E1809381000C941A
:1005C000D02281110BC080918000877F80938000B2
:1005D00010928D0010928C002F9808952F988330E0
:1005E00041F4809180008860809380008FEF9FEFBE
:1005F00012C09091800098609093800023E030E0DA
:10060000281B3109220F331F8FEF9FEF02C09695F1
:1006100087952A95E2F790938D0080938C0008953A
:100620008B3B910568F4883A910530F5853A910540
:10063000C0F48430910598F4019709F06FC071C03F
:10064000803E910508F46AC0883E910540F09C0107
:10065000205F31092031310508F060C05CC09C0189
:10066000A1C0853A910509F45FC0863A910509F465
:100670005EC023E830E496C0883A910509F45AC078
:10068000893A910509F459C08A3A910509F458C08C
:100690008B3A910509F457C08C3A910509F456C07C
:1006A0008D3A910509F455C0803B910509F454C079
:1006B0008E3A910509F453C08F3A910509F452C05E
:1006C000813B910509F451C0823B910509F450C06A
:1006D000833B910509F44FC0843B910509F44EC05A
:1006E000853B910509F44DC0863B910509F44CC04A
:1006F000873B910509F44BC0883B910509F44AC03A
:10070000893B910509F449C08A3B910509F048C02D
:100710002AE236E447C09C01306544C020E030E066
:1007200041C021E030E03EC021E830E43BC022E897
:1007300030E438C022EE34E435C029EE34E432C06F
:100740002AEE34E42FC025EB34E42CC026EB34E44D
:1007500029C027EB34E426C02CEC34E423C02DEC74
:1007600034E420C023E835E41DC02AE835E41AC08B
:1007700022E935E417C024E935E414C021E236E467
:1007800011C023E236E40EC024E236E40BC025E2B9
:1007900036E408C026E236E405C027E236E402C0AB
:1007A00020E034E4C901089508959CE0799FF001A8
:1007B00011249CE3899FE00DF11D1124E60FF11D2A
:1007C000EE0FFF1FE455FF4F25913491C9010895A5
:1007D000880F991F845D9040FC0125913491C901D7
:1007E0000895880F991F84559F4FFC0125913491DE
:1007F000C90108950E94D5039C019A9581159F41D6
:1008000010F4C9010895C90190528115904128F44E
:10081000C9019F700E94F1030895C9019053811589
:10082000904120F4C9019927906C0895C901905412
:10083000409728F4C9018F709927946D089520314D
:1008400080E4380719F480E091ED0895213190E4B7
:10085000390719F480E090ED0895223140E434071F
:1008600019F480E092ED0895233180E4380719F4FB
:1008700080E093ED0895211590E5390769F40E9411
:1008800015162FEF44E38CE0215040408040E1F703
:1008900000C000000C94BD1C213090E5390731F4F4
:1008A0008091D00181608093D0010895C901905555
:1008B0008115904108F062C0432F55274F7055278E
:1008C00041305105F9F4C90174E0880F991F7A95F8
:1008D000E1F788279370B901E3E0660F771FEA9587
:1008E000E1F760767727862B972B9C682370332758
:1008F00002C0440F551F2A95E2F74F715527842BEC
:10090000952B08954230510529F4922F8827816F45
:10091000906A089543305105B9F4C90153E0880F36
:10092000991F5A95E1F7807E97702370332741E035
:1009300050E002C0440F551F2A95E2F74F7155272A
:10094000842B952B9C6808954430510549F5C901C5
:1009500043E0880F991F4A95E1F7807E97702370D6
:10096000332741E050E002C0440F551F2A95E2F7BB
:100970004F715527842B952B9A680895C90190577C
:100980008115904120F4C9019F7090620895C901BA
:1009900090588115904120F4C9019F70906A089584
:1009A000203E3105E0F4203C310568F52133310566
:1009B00009F475C048F42932310509F46BC02A32B4
:1009C000310509F07BC075C02933310501F12238AA
:1009D0003105E9F02533310509F070C051C0233EDF
:1009E0003105B1F140F4203E3105D1F0223E310510
:1009F00009F064C01CC0263E310579F1273E31055F
:100A000009F05CC038C0C9010E94E80308958091D4
:100A1000E10180FD02C081FF51C080EE90E04FC037
:100A20008091E10180FFF9CF89E390E048C0809197
:100A3000E10182FF0AC08091E10184FF03C080E0F0
:100A400090E03DC083EE90E03AC082EE90E037C087
:100A50008091E10182FFEFCFF8CF8091E10183FF28
:100A600007C08091E10184FDEACF87EE90E027C0C6
:100A700086EE90E024C08091E10183FFF2CFF8CFB1
:100A80008091E10185FF03C089E290E018C085E311
:100A900090E015C08091E10185FDF9CFF5CF8091FF
:100AA000E10186FF03C08AE290E009C081E390E0A3
:100AB00006C08091E10186FDF9CFF5CFC9010E9402
:100AC0001003089508955F926F927F928F929F9284
:100AD000AF92BF92CF92DF92EF92FF920F931F934C
:100AE000CF93DF93CDB7DEB72A970FB6F894DEBF6A
:100AF0000FBECDBF9E012F5F3F4F4E018BE0880E92
:100B0000911C60E070E000E010E0E12CF12CC12CC1
:100B1000D12CA12CB12C8AE0782E622E532E41E0EC
:100B200050E0E4E1F1E0A62DB52D872D01900D9266
:100B30008A95E1F7F901819191919F01FC01E07F94
:100B4000FF27E032F10559F48F709927FA0102C0AE
:100B5000EE0FFF1F8A95E2F7AE2ABF2A37C0E033B7
:100B6000F10559F48F709927FA0102C0EE0FFF1FAB
:100B70008A95E2F7CE2ADF2A29C0E034F10559F43C
:100B80008F709927FA0102C0EE0FFF1F8A95E2F7D6
:100B9000EE2AFF2A1BC0E035F10559F48F70992722
:100BA000FA0102C0EE0FFF1F8A95E2F70E2B1F2BF2
:100BB0000DC0E036F10551F48F709927FA0102C09B
:100BC000EE0FFF1F8A95E2F76E2B7F2B2815390554
:100BD00009F0A7CF94B18A2D8095892384B985B176
:100BE0008A2985B997B18C2D8095892387B988B1D9
:100BF0008C2988B99AB18E2D809589238AB98BB1B9
:100C00008E298BB99DB1802F809589238DB98EB1A6
:100C1000802B8EB990B3862F8095892380BB81B3BA
:100C2000862B81BB2A960FB6F894DEBF0FBECDBFD0
:100C3000DF91CF911F910F91FF90EF90DF90CF90B8
:100C4000BF90AF909F908F907F906F905F9008952E
:100C50005F926F927F928F929F92AF92BF92CF924C
:100C6000DF92EF92FF920F931F93CF93DF93CDB755
:100C7000DEB768970FB6F894DEBF0FBECDBF85B75D
:100C8000806885BF85B7806885BF0E9463059E0127
:100C90002F5F3F4F4E0189E1880E911C60E070E0AC
:100CA00000E010E0E12CF12CC12CD12CA12CB12CB6
:100CB00098E1792E622E532E41E050E0EEE1F1E012
:100CC000A62DB52D872D01900D928A95E1F7F9019A
:100CD000819191919F01FC01E07FFF27E032F105B6
:100CE00059F48F709927FA0102C0EE0FFF1F8A9501
:100CF000E2F7AE2ABF2A37C0E033F10559F48F700E
:100D00009927FA0102C0EE0FFF1F8A95E2F7CE2A5B
:100D1000DF2A29C0E034F10559F48F709927FA01D0
:100D200002C0EE0FFF1F8A95E2F7EE2AFF2A1BC0D2
:100D3000E035F10559F48F709927FA0102C0EE0FE2
:100D4000FF1F8A95E2F70E2B1F2B0DC0E036F10531
:100D500051F48F709927FA0102C0EE0FFF1F8A9598
:100D6000E2F76E2B7F2B2815390509F0A7CF94B138
:100D70008A2D8095892384B985B18A2985B997B14F
:100D80008C2D8095892387B988B18C2988B99AB12F
:100D90008E2D809589238AB98BB18E298BB99DB10F
:100DA000802F809589238DB98EB1802B8EB990B319
:100DB000862F8095892380BB81B3862B81BB1092BF
:100DC00055011092540110925F0110925E01109231
:100DD0005701109256011092610110926001109219
:100DE0005901109258011092630110926201109201
:100DF0005B0110925A0110926501109264011092E9
:100E00005D0110925C0110926701109266018FEBF8
:100E100092E0892BB9F068960FB6F894DEBF0FBE4A
:100E2000CDBFDF91CF911F910F91FF90EF90DF9099
:100E3000CF90BF90AF909F908F907F906F905F907A
:100E40000C94BF0268960FB6F894DEBF0FBECDBFFC
:100E5000DF91CF911F910F91FF90EF90DF90CF9096
:100E6000BF90AF909F908F907F906F905F9008950C
:100E70005F926F927F928F929F92AF92BF92CF922A
:100E8000DF92EF92FF920F931F93CF93DF93CDB733
:100E9000DEB7A2970FB6F894DEBF0FBECDBF7E01BE
:100EA00049E1E40EF11C2EE5C22E21E0D22E5E01B6
:100EB00053E2A50EB11C3AE0532E470101E010E0C9
:100EC00048E1642E55E0752EE4E1F1E0D401852D72
:100ED00001900D928A95E1F7F701819191917F013F
:100EE0009C01207F33272032310589F424B18F7093
:100EF0009927A80102C0440F551F8A95E2F7CA013D
:100F0000242B24B995B18095892385B94FC020330E
:100F1000310589F427B18F709927F80102C0EE0FCF
:100F2000FF1F8A95E2F7CF012E2B27B998B1809544
:100F3000892388B93BC02034310589F42AB18F70E8
:100F40009927A80102C0440F551F8A95E2F7CA01EC
:100F5000242B2AB99BB1809589238BB927C02035D2
:100F6000310589F42DB18F709927F80102C0EE0F79
:100F7000FF1F8A95E2F7CF012E2B2DB99EB18095E8
:100F800089238EB913C02036310581F420B38F70C8
:100F90009927A80102C0440F551F8A95E2F7CA019C
:100FA000242B20BB91B38095892381BB50EA5A95AD
:100FB000F1F7BE016F5F7F4F80E090E020E030E00E
:100FC000EEE1F1E0DE011196462D01900D924A9579
:100FD000E1F7FB0141915191BF01FA01E07FFF2749
:100FE000E032F10511F4E3B113C0E033F10511F47F
:100FF000E6B10EC0E034F10511F4E9B109C0E03505
:10100000F10511F4ECB104C0E036F105B9F4EFB12B
:10101000F0E04F70552702C0F595E7954A95E2F745
:10102000E0FD08C0A801022E02C0440F551F0A941B
:10103000E2F702C040E050E0842B952B2F5F3F4F3A
:101040002C30310509F0BCCFF60120813181281701
:10105000390721F091838083709200010E9463051B
:10106000F2E0CF0ED11CEA14FB0409F02DCF8091E1
:1010700000018823A1F1815080930001882339F079
:101080008FE99FE00197F1F700C0000028C0809130
:101090005E0190915F01909355018093540180917E
:1010A0006001909161019093570180935601809166
:1010B000620190916301909359018093580180914E
:1010C00064019091650190935B0180935A01809136
:1010D00066019091670190935D0180935C018AECB9
:1010E00092E0892B11F00E94CA0281E0A2960FB60D
:1010F000F894DEBF0FBECDBFDF91CF911F910F914E
:10110000FF90EF90DF90CF90BF90AF909F908F9027
:101110007F906F905F900895E82FF0E0EE0FFF1F33
:10112000EC5AFE4F8081918108950895809171015C
:101130000895CF93DF9300D01F92CDB7DEB72091F3
:10114000E701243021F523E029839B838A832093C0
:10115000E9008FEF06C095ED9A95F1F7000088231E
:1011600029F09091E800815095FFF5CF8091E8003B
:1011700085FF0DC040E050E063E070E0CE010196D5
:101180000E94280B8091E8008E778093E8000F90F2
:101190000F900F90DF91CF910895CF93DF9300D000
:1011A0001F92CDB7DEB72091E701243029F522E068
:1011B00029839B838A8383E08093E9008FEF06C0B5
:1011C00095ED9A95F1F70000882329F09091E800B9
:1011D000815095FFF5CF8091E80085FF0DC040E07C
:1011E00050E063E070E0CE0101960E94280B8091F0
:1011F000E8008E778093E8000F900F900F90DF91BA
:10120000CF9108952091E7012430F9F422E0209352
:10121000E9002FEF06C035ED3A95F1F700002223E3
:1012200029F03091E800215035FFF5CF2091E800FA
:1012300025FF0BC040E050E065E070E00E94280B05
:101240008091E8008E778093E8000895CF93DF9334
:10125000EC018091E701843041F581E08093E90061
:101260008FEF06C095ED9A95F1F70000882329F0DD
:101270009091E800815095FFF5CF8091E80085FFBF
:1012800014C040E050E068E070E0CE010E94280BFE
:101290008091E8008E778093E80088E0FE01A9E65F
:1012A000B1E001900D928A95E1F7DF91CF91089519
:1012B0008091E601811109C00E94C80C0E94250D91
:1012C0008091E20084608093E20008951092E6012C
:1012D0000895089508950C94201C809172018F5FE9
:1012E0008093720162E30E948924911135C01092AB
:1012F000720180917301882379F18091E701843034
:1013000049F58091E9008F709091EC0090FF02C048
:1013100090E801C090E0982B84E08093E9008091F0
:10132000EB0080FF14C08091EE0087FD03C00FC06A
:101330001092F1008091E80085FDFACF8091E800DD
:1013400080FF05C08091E8008E778093E8009F7051
:101350009093E90010927301089542E061EC81E0FE
:101360000E943E0C42E061EC82E00E943E0C42E0B2
:1013700061EC83E00E943E0C42E261EC84E00C945C
:101380003E0C8091E901833009F454C030F481307F
:1013900071F0823009F0A5C08CC08A3009F479C0A0
:1013A0008B3009F45FC0893009F09BC020C0809168
:1013B000E801813A09F095C08091E800877F809329
:1013C000E8008091EC019091ED01892B21F060E023
:1013D00080E090E003C068E089E691E070E00E9460
:1013E000770B8091E8008B778093E80008958091D7
:1013F000E801813209F075C08091EC019091ED0116
:10140000892B09F06EC08091E800877F8093E80007
:1014100005C08091E701882309F463C08091E8004A
:1014200082FFF7CF8091F100809371018091E800F5
:101430008B7753C08091E801813A09F052C08091C6
:10144000EC019091ED01892B09F04BC08091E800EF
:10145000877F8093E8008091E80080FFFCCF809137
:101460000B0136C08091E8018132D9F58091EC0101
:101470009091ED01892BA9F58091E800877F8093F9
:10148000E8000E94750C8091EA0180930B010C9496
:1014900015168091E801813221F58091E800877F5F
:1014A0008093E8000E94750C8091EB0180936801A5
:1014B00008958091E801813AA1F48091E800877F46
:1014C0008093E8008091E80080FFFCCF8091680164
:1014D0008093F1008091E8008E778093E8000C946F
:1014E000750C089584B7877F84BF88E10FB6F894A0
:1014F00080936000109260000FBE90E080E80FB60D
:10150000F89480936100909361000FBE0E943310A5
:101510000E94C80C0E94250D8091E2008460809397
:10152000E20078940E94C20F0E94351081E091E0A1
:101530000E94DF0F0BC00E94DD1B8091E501882314
:1015400029F00E94081C81110E94120B8091E70172
:10155000853089F30E943F10F9CF292F332723309C
:101560003105B1F04CF42130310509F44DC0223081
:10157000310509F04EC007C02132310541F1223258
:10158000310591F146C0E4E7F0E082E693E045C022
:1015900099278130910569F08230910589F0892B76
:1015A00009F037C0EEE5F3E0E491F0E08EE593E07A
:1015B00034C0E0E3F3E0E491F0E080E393E02DC099
:1015C000E4E0F3E0E491F0E084E093E026C06430EE
:1015D00000F5E62FF0E0EE0FFF1FEA5CFE4F808182
:1015E0009181E9E0F0E019C0643098F4E62FF0E072
:1015F000DF01AA0FBB1FA25CBE4F8D919C91EA5BDD
:10160000FE4FE081F0E009C0E2E1F0E086ED93E01A
:1016100004C0E0E0F0E080E090E0DA018D939C937C
:10162000CF01089580E189BD82E189BD09B400FE42
:10163000FDCF8091D8008F7D8093D8008091E0000D
:1016400082608093E0008091E00081FDFCCF0895EE
:10165000BF92CF92DF92EF92FF920F931F93CF939F
:10166000DF937C018B01EA010E94960CB82E811158
:1016700033C0209731F028813981021B130BE20E11
:10168000F31EC12CD12C23C08091E80085FD15C02C
:101690008091E8008E778093E800209749F0888158
:1016A00099818C0D9D1D9983888325E0B22E14C0ED
:1016B0000E94960C882359F00EC0F70181917F019A
:1016C0008093F10001501109FFEFCF1ADF0A0115D5
:1016D0001105D1F601C0B82E8B2DDF91CF911F914E
:1016E0000F91FF90EF90DF90CF90BF9008954091C1
:1016F000EE015091EF014617570748F0611571054B
:1017000039F44091E8004E774093E80001C0BA01F7
:10171000FC0140E033C08091E701882309F444C014
:10172000853009F443C08091E80083FD41C0809179
:10173000E80082FD33C08091E80080FF1FC09091D7
:10174000F3008091F200392F20E0A901482BCA0153
:1017500006C041914093F1006150710901966115F5
:10176000710519F088309105A0F341E0089709F060
:1017700040E08091E8008E778093E8006115710564
:1017800051F64111C8CF0AC08091E701882361F06A
:10179000853061F08091E80083FD0AC08091E80007
:1017A00082FFF2CF80E0089582E0089583E00895FB
:1017B00081E008954091EE015091EF0146175707DF
:1017C00048F06115710539F44091E8004E77409377
:1017D000E80001C0BA01FC0140E034C08091E7019B
:1017E000882309F445C0853009F444C08091E8009D
:1017F00083FD42C08091E80082FD34C08091E80002
:1018000080FF20C09091F3008091F200392F20E0FA
:10181000A901482BCA0107C044914093F1003196B9
:101820006150710901966115710519F088309105B3
:1018300098F341E0089709F040E08091E8008E7746
:101840008093E8006115710549F64111C7CF0AC0C0
:101850008091E701882361F0853061F08091E80094
:1018600083FD0AC08091E80082FFF2CF80E00895F6
:1018700082E0089583E0089581E00895982F2CC0B8
:101880009093E900981739F07091EC002091ED00E9
:101890005091F00003C0242F762F50E021FD02C0AC
:1018A0009F5F1AC03091EB003E7F3093EB00309188
:1018B000ED003D7F3093ED003091EB0031603093CF
:1018C000EB007093EC002093ED005093F00020911A
:1018D000EE0027FDE5CF07C0973090F28F70809320
:1018E000E90081E0089580E008958091E80187FD96
:1018F00005C08091E80080FF0EC012C08091E80012
:1019000082FD05C08091E7018111F8CF0895809193
:10191000E8008B7708C08091E7018111EACF089534
:101920008091E8008E778093E80008958091E4002C
:101930009091E50045E62091EC0020FD1FC023C0FA
:101940002091E701222391F0253091F02091EB00C6
:1019500025FD10C02091E4003091E50028173907DB
:1019600051F34150C90139F784E0089582E00895A8
:1019700083E0089581E0089580E008952091E800D3
:1019800020FFDECFF9CF2091E80022FFD9CFF4CF9E
:101990000E94360D0E943E0DE0EEF0E080818160F5
:1019A0008083E8EDF0E080818F77808319BCA7ED1C
:1019B000B0E08C918E7F8C9380818F7E808310929B
:1019C000E60108950F931F93CF93DF930E94360D86
:1019D0000E943E0DC8EDD0E088818F778883888192
:1019E0008068888388818F7D888319BC1092E70185
:1019F0001092E3011092E5011092E40100EE10E074
:101A0000F80180818B7F808388818160888342E0B8
:101A100060E080E00E943E0CE1EEF0E080818E7F8D
:101A20008083E2EEF0E08081816080838081886045
:101A30008083F80180818E7F8083888180618883A4
:101A4000DF91CF911F910F910895E8EDF0E0808133
:101A50008F7E8083E7EDF0E080818160808384E089
:101A600082BF81E08093E6010C94E20CE8EDF0E0A7
:101A700080818E7F80831092E20008951092DA00B8
:101A80001092E10008951F920F920FB60F92112449
:101A90002F933F934F935F936F937F938F939F9376
:101AA000AF93BF93EF93FF938091E10082FF0BC050
:101AB0008091E20082FF07C08091E1008B7F8093DC
:101AC000E1000E946D098091DA0080FF1FC08091C3
:101AD000D80080FF1BC08091DA008E7F8093DA00EF
:101AE0008091D90080FF0DC080E189BD82E189BD70
:101AF00009B400FEFDCF81E08093E7010E94580900
:101B000005C019BC1092E7010E9466098091E100AE
:101B100080FF19C08091E20080FF15C08091E20033
:101B20008E7F8093E2008091E20080618093E200EA
:101B30008091D80080628093D80019BC85E08093A2
:101B4000E7010E946A098091E10084FF30C0809122
:101B5000E20084FF2CC080E189BD82E189BD09B427
:101B600000FEFDCF8091D8008F7D8093D8008091BA
:101B7000E1008F7E8093E1008091E2008F7E809370
:101B8000E2008091E20081608093E2008091E301B5
:101B9000882311F084E007C08091E30087FF02C032
:101BA00083E001C081E08093E7010E946B0980918E
:101BB000E10083FF29C08091E20083FF25C080916E
:101BC000E100877F8093E10082E08093E70110923B
:101BD000E3018091E1008E7F8093E1008091E2003B
:101BE0008E7F8093E2008091E20080618093E2002A
:101BF00042E060E080E00E943E0C8091F00088604E
:101C00008093F0000E946909FF91EF91BF91AF911D
:101C10009F918F917F916F915F914F913F912F9104
:101C20000F900FBE0F901F9018951F920F920FB636
:101C30000F9211242F933F934F935F936F937F9352
:101C40008F939F93AF93BF93CF93EF93FF93809125
:101C5000E9008F709091EC0090FF02C090E801C005
:101C600090E0C92FC82B1092E9008091F000877F87
:101C70008093F00078940E94590E1092E9008091B0
:101C8000F00088608093F000CF70C093E900FF916E
:101C9000EF91CF91BF91AF919F918F917F916F9174
:101CA0005F914F913F912F910F900FBE0F901F901A
:101CB00018951F93CF93DF93CDB7DEB7AC970FB6D0
:101CC000F894DEBF0FBECDBFE8EEF1E08091F100E9
:101CD000819321E0E03FF207C9F70E94C10980919A
:101CE000E80083FF37C18091E8019091E9019530C8
:101CF00009F488C038F49130B1F170F0933009F0F4
:101D000029C131C0983009F4F8C0993009F404C1F0
:101D1000963009F01FC19DC0803821F0823809F04B
:101D200019C108C08091E4019091E501992389F0DF
:101D300082600FC08091EC019091ED018F70992726
:101D40008093E9008091EB0085FB882780F9109251
:101D5000E9009091E800977F9093E8008093F1006C
:101D60001092F100D5C0882319F0823009F0F2C03A
:101D70008F7121F0823009F0EDC00BC08091EA0133
:101D8000813009F0E7C0933009F080E08093E501ED
:101D90002FC08091EA0181112BC08091EC019091BC
:101DA000ED018F709927009709F4D4C08093E90062
:101DB0002091EB0020FF1CC02091E901233021F489
:101DC0008091EB00806212C09091EB009061909343
:101DD000EB0021E030E001C0220F8A95EAF7209362
:101DE000EA001092EA008091EB0088608093EB009B
:101DF0001092E9008091E800877F8093E8000E94BC
:101E0000750CA8C08111A6C08091EA019091EB01E8
:101E10008F779927182F9091E3009078982B9093C3
:101E2000E3008091E800877F8093E8000E94750CB2
:101E30008091E80080FFFCCF8091E3008068809370
:101E4000E300112311F083E001C082E08093E701F9
:101E500081C08058823008F07DC08091EA01909165
:101E6000EB018C3D23E0920779F583E08A838AE2D7
:101E700089834FB7F894DE01139620E03EE051E2EB
:101E8000E32FF0E050935700E49120FF03C0E29568
:101E9000EF703F5FEF708E2F90E0EA3010F0C79642
:101EA00001C0C0968D939D932F5F243149F74FBF9A
:101EB0008091E800877F8093E8006AE270E0CE01BD
:101EC00001960E94770B13C0AE01455D5F4F609194
:101ED000EC010E94AD0A0097E9F12091E800277F0C
:101EE0002093E800BC018BA59CA50E94DA0B809191
:101EF000E8008B778093E8002DC0803859F58091F9
:101F0000E800877F8093E8008091E3018093F100EF
:101F10008091E8008E7771CF81111CC09091EA0109
:101F20009230C0F48091E800877F8093E80090931E
:101F3000E3010E94750C8091E301811104C080913E
:101F4000E30087FF02C084E001C081E08093E701E5
:101F50000E94AD098091E80083FF0AC08091E800EB
:101F6000877F8093E8008091EB0080628093EB0094
:101F7000AC960FB6F894DEBF0FBECDBFDF91CF9108
:101F80001F910895CF938091E7018823B1F080914C
:101F9000E9008F709091EC0090FF02C090E801C0C2
:101FA00090E0C92FC82B1092E9008091E80083FDD2
:101FB0000E94590ECF70C093E900CF91089590937D
:101FC0007501809374010895E0917401F091750199
:101FD000309721F00190F081E02D099480E0089580
:101FE000E0917401F0917501309721F00280F38146
:101FF000E02D09940895E0917401F09175013097F6
:1020000021F00480F581E02D099408952091760156
:10201000309177018217930771F090937701809345
:102020007601E0917401F0917501309721F00680FE
:10203000F781E02D0994089520917801309179017C
:102040008217930771F09093790180937801E09162
:102050007401F0917501309721F00084F185E02D35
:102060000994089508950C9432100E94541C0E9403
:1020700028060E94281D0C94D0220C9462055F92C1
:102080006F927F928F929F92AF92BF92CF92DF9288
:10209000EF92FF920F931F93CF93DF93CDB7DEB7ED
:1020A0002A970FB6F894DEBF0FBECDBF0E94380747
:1020B0009AE7C92E91E0D92E00E010E0AA24A3945B
:1020C000B12C502E802F0E948C083C01F601E1902B
:1020D000F1906F01E826F926E114F10431F40F5F65
:1020E0001F4F0530110569F73AC08091D00181FD7D
:1020F0000E94950820E030E04501022E02C0880CC5
:10210000991C0A94E2F7C4018E219F21892B09F1C1
:102110002E835F826820792081E0672809F480E0BF
:1021200088870E945D1C8160782F9A8789874E81FD
:102130005F8168858A850E94F810F801EE0FFF1F05
:10214000E658FE4F8081918188259925918380836F
:1021500016C02F5F3F4F2C30310571F6C0CF8FEF87
:1021600089838A831B820E945D1C8160782F9D83F6
:102170008C8349815A816B818D810E94F8100E9465
:102180001520109184010E94E40F1817D9F00E94C5
:10219000E40F809384012A960FB6F894DEBF0FBE39
:1021A000CDBFDF91CF911F910F91FF90EF90DF9006
:1021B000CF90BF90AF909F908F907F906F905F90E7
:1021C0000C943D102A960FB6F894DEBF0FBECDBF1B
:1021D000DF91CF911F910F91FF90EF90DF90CF9003
:1021E000BF90AF909F908F907F906F905F90089579
:1021F000CF93DF93CDB7DEB72B970FB6F894DEBF42
:102200000FBECDBF4F83588769877A878B87DE01E2
:10221000119686E0FD0111928A95E9F785E0FE01AD
:10222000379601900D928A95E1F749815A816B8129
:102230007C818D819E810E94D4182B960FB6F894D4
:10224000DEBF0FBECDBFDF91CF910895CF93C82FD2
:10225000882309F4C1C0823859F40E94E40F81FD3B
:10226000BBC089E30E943B1B0E94B71B89E30CC0E3
:10227000833879F40E94E40F80FDAEC083E50E94AC
:102280003B1B0E94B71B83E50E945D1BCF910C9402
:10229000B71B843859F40E94E40F82FD9DC087E487
:1022A0000E943B1B0E94B71B87E4EECF8450813A0B
:1022B00048F48C2F0E94322281118EC08C2F0E94F4
:1022C0003B1BE4CF8C2F805E883050F4C77081E0D8
:1022D00090E001C0880FCA95EAF70E947E1BD6CF16
:1022E0008C2F855A833078F4C53A29F0C63A31F4F8
:1022F00082E890E005C081E890E002C083E890E0C9
:10230000CF910C9406108C2F885A833108F064C04A
:10231000C83A39F1C93A41F1CA3A49F1CB3A51F1D7
:10232000CC3A59F1CD3A61F1C03B69F1CE3A71F145
:10233000CF3A79F1C13B81F1C23B89F1C33B91F1C5
:10234000C43B99F1C53BA1F1C63BA9F1C73BB1F133
:10235000C83BB9F1C93BC1F1CA3BC9F58AE292E079
:1023600038C082EE90E035C089EE90E032C08AEE4F
:1023700090E02FC085EB90E02CC086EB90E029C068
:1023800087EB90E026C08CEC90E023C08DEC90E0D1
:1023900020C083E891E01DC08AE891E01AC082E97C
:1023A00091E017C084E991E014C081E292E011C08D
:1023B00083E292E00EC084E292E00BC085E292E0FC
:1023C00008C086E292E005C087E292E002C080E0A9
:1023D00090E0CF910C941C10CF910895882309F4BC
:1023E0004DC0823859F40E94E40F81FF47C089E351
:1023F0000E943B1B0E94B71B89E30CC0833871F419
:102400000E94E40F80FF3AC083E50E943B1B0E94BC
:10241000B71B83E50E945D1B0C94B71B843859F4ED
:102420000E94E40F82FF2AC087E40E943B1B0E94A7
:10243000B71B87E4EFCF982F9450913A08F4EACF76
:10244000982F905E983058F4282F277081E090E004
:1024500001C0880F2A95EAF70E94841BDDCF982FD0
:10246000955A933020F480E090E00C940610885A3E
:10247000833120F480E090E00C941C1008958823B0
:1024800021F00E947E1B0C94B71B0895882321F035
:102490000E94841B0C94B71B0895BF92CF92DF92C9
:1024A000EF92FF920F931F93CF93DF93CDB7DEB7D9
:1024B00027970FB6F894DEBF0FBECDBF8C0185E025
:1024C000F801DE01119601900D928A95E1F7F8016D
:1024D00030812181F280558152955F708381948192
:1024E000892B39F02F3F41F481E090E03F3F31F0FC
:1024F00003C081E090E002C080E090E080FD73C303
:1025000039832A8389819A815E830E94F81AB92EC1
:102510008F830E94F71A0E941F1A2B2D22952F706D
:1025200030E05E816F812530310509F4E6C06CF43E
:10253000243031050CF0A2C04B2D407F8B2D8F70C5
:10254000223031050CF045C017C02C3031054CF459
:102550002A3031050CF0E7C12830310509F043C3BA
:10256000E5C02D30310509F4BAC20CF4A2C22F30F7
:10257000310509F038C323C3182F411101C002C02F
:102580001295107FFF2059F0112309F46BC2812F9F
:102590006F830E948E1B0E94B71B6F8163C2862FC0
:1025A0000E94EE11112309F41EC3812F0E94941B77
:1025B00027960FB6F894DEBF0FBECDBFDF91CF9147
:1025C0001F910F91FF90EF90DF90CF90BF900C94F0
:1025D000B71B403211F08295807F662319F061307D
:1025E00071F523C0FF20B1F0511101C032C051304C
:1025F00081F527960FB6F894DEBF0FBECDBFDF91F1
:10260000CF911F910F91FF90EF90DF90CF90BF90EF
:102610000C949E1B511101C003C0513009F4E3C258
:102620008E830E94A11B8E819AC1FF2021F056301B
:1026300008F0D9C20EC0553008F0D5C290C1FF20B5
:10264000C9F0552331F0F801958190FF0BC29F70BE
:10265000958327960FB6F894DEBF0FBECDBFDF91EE
:10266000CF911F910F91FF90EF90DF90CF90BF908F
:102670000C943F12552309F472C109C22B2D2695E3
:102680002695237030E02115310529F021303105E0
:1026900009F0A9C219C0FF2021F0862F9B2D93704D
:1026A00002C080E090E027960FB6F894DEBF0FBE20
:1026B000CDBFDF91CF911F910F91FF90EF90DF90F1
:1026C000CF90BF900C940610FF2021F0862F9B2DF9
:1026D000937002C080E090E027960FB6F894DEBFBA
:1026E0000FBECDBFDF91CF911F910F91FF90EF9063
:1026F000DF90CF90BF900C941C10862FFF2019F014
:102700000E941B1F02C00E94831F27960FB6F894D9
:10271000DEBF0FBECDBFDF91CF911F910F91FF9014
:10272000EF90DF90CF90BF900C940A208B2D837098
:1027300009F079C0F11057C2262F229526952770EF
:10274000220F220F862F8F70C82ED12CE12CF12C56
:10275000022E04C0CC0CDD1CEE1CFF1C0A94D2F728
:1027600064FF10C06FE070E080E090E004C0660F8E
:10277000771F881F991F2A95D2F7609570958095CD
:10278000909503C060E070E0CB012B2D2695269537
:102790002370422F50E042305105D9F043305105AB
:1027A00069F16C297D298E299F294130510551F10C
:1027B00027960FB6F894DEBF0FBECDBFDF91CF9145
:1027C0001F910F91FF90EF90DF90CF90BF900C94EE
:1027D000341A6C297D298E299F2927960FB6F894E3
:1027E000DEBF0FBECDBFDF91CF911F910F91FF9044
:1027F000EF90DF90CF90BF900C94461A0E94341A4D
:10280000C701B60127960FB6F894DEBF0FBECDBF45
:10281000DF91CF911F910F91FF90EF90DF90CF90BC
:10282000BF900C94221AFF2019F08B2D817001C0EB
:102830008695882309F4D7C1262F229526952770DF
:10284000220F220F862F8F70C82ED12CE12CF12C55
:10285000022E04C0CC0CDD1CEE1CFF1C0A94D2F727
:1028600064FF10C06FE070E080E090E004C0660F8D
:10287000771F881F991F2A95D2F7609570958095CC
:10288000909503C060E070E0CB012B2D2695269536
:102890002370422F50E042305105D9F043305105AA
:1028A00069F16C297D298E299F294130510551F10B
:1028B00027960FB6F894DEBF0FBECDBFDF91CF9144
:1028C0001F910F91FF90EF90DF90CF90BF900C94ED
:1028D000D31A6C297D298E299F2927960FB6F89443
:1028E000DEBF0FBECDBFDF91CF911F910F91FF9043
:1028F000EF90DF90CF90BF900C94E51A0E94D31A0E
:10290000C701B60127960FB6F894DEBF0FBECDBF44
:10291000DF91CF911F910F91FF90EF90DF90CF90BB
:10292000BF900C94C11A603F59F120F4603E08F446
:1029300094C008C0623F09F467C0F0F1633F09F03A
:102940008CC065C0162F1F708B2D8F71FF2021F05A
:102950000E946C1A812F7DCE0E94871A812F2796A4
:102960000FB6F894DEBF0FBECDBFDF91CF911F91A0
:102970000F91FF90EF90DF90CF90BF900C94461294
:10298000FF20B1F0553008F02EC18B2D8F712796A6
:102990000FB6F894DEBF0FBECDBFDF91CF911F9170
:1029A0000F91FF90EF90DF90CF90BF900C94A61AFC
:1029B000563008F018C1E9CFFF2099F08B2D8F71A8
:1029C00027960FB6F894DEBF0FBECDBFDF91CF9133
:1029D0001F910F91FF90EF90DF90CF90BF900C94DC
:1029E0006C1A8B2D8F7127960FB6F894DEBF0FBE31
:1029F000CDBFDF91CF911F910F91FF90EF90DF90AE
:102A0000CF90BF900C94871AF110EBCFD7CFFF2057
:102A100099F08B2D8F7127960FB6F894DEBF0FBEFD
:102A2000CDBFDF91CF911F910F91FF90EF90DF907D
:102A3000CF90BF900C945D1A27960FB6F894DEBF26
:102A40000FBECDBFDF91CF911F910F91FF90EF90FF
:102A5000DF90CF90BF900C94581AFF20A9F0552317
:102A600009F4ACCF862F27960FB6F894DEBF0FBEC1
:102A7000CDBFDF91CF911F910F91FF90EF90DF902D
:102A8000CF90BF900C942611552309F4AACF862F1E
:102A900027960FB6F894DEBF0FBECDBFDF91CF9162
:102AA0001F910F91FF90EF90DF90CF90BF900C940B
:102AB000EE114B2D4F70C8010E94AB0227960FB646
:102AC000F894DEBF0FBECDBFDF91CF911F910F9164
:102AD000FF90EF90DF90CF90BF900C948A19F11087
:102AE00082C09B2D9F70492F50E04230510599F1D3
:102AF00044F44115510569F04130510509F073C0A6
:102B000019C043305105C1F14430510509F06BC083
:102B100044C027960FB6F894DEBF0FBECDBFDF913D
:102B2000CF911F910F91FF90EF90DF90CF90BF90CA
:102B30000C94E12227960FB6F894DEBF0FBECDBFEE
:102B4000DF91CF911F910F91FF90EF90DF90CF9089
:102B5000BF900C94F82227960FB6F894DEBF0FBEF4
:102B6000CDBFDF91CF911F910F91FF90EF90DF903C
:102B7000CF90BF900C94142327960FB6F894DEBF25
:102B80000FBECDBFDF91CF911F910F91FF90EF90BE
:102B9000DF90CF90BF900C942723862F27960FB6F7
:102BA000F894DEBF0FBECDBFDF91CF911F910F9183
:102BB000FF90EF90DF90CF90BF900C944B234B2D64
:102BC0004F70C80127960FB6F894DEBF0FBECDBF79
:102BD000DF91CF911F910F91FF90EF90DF90CF90F9
:102BE000BF900C94D40327960FB6F894DEBF0FBEA7
:102BF000CDBFDF91CF911F910F91FF90EF90DF90AC
:102C0000CF90BF9008950E949B1B0E94701B0E9452
:102C1000B71B0E94B6200E940A2080E090E00E942C
:102C2000061080E090E00C941C100E948B1B0C940A
:102C300003160E94F81A292F22952F7030E02C30AD
:102C400031054CF42A3031056CF422503109223020
:102C5000310590F407C02C30310551F02F3031058B
:102C600059F406C0803E10F0803F31F481E00895B1
:102C700093FB882780F9089580E00895CF93DF9330
:102C800000D000D01F92CDB7DEB70F900F900F90FD
:102C90000F900F90DF91CF910895CF93DF9300D0E5
:102CA00000D000D0CDB7DEB726960FB6F894DEBFC1
:102CB0000FBECDBFDF91CF9108951F93CF93DF93C8
:102CC000C091BB0116E012C0D0E01C9FF0011D9F17
:102CD000F00D1124E557FE4F4081518162817381CF
:102CE000848195810E944D162196C7708091BC0108
:102CF000C813EACFDF91CF911F91089540918501CC
:102D000050918601609187017091880180918901BD
:102D100090918A010C944D160F931F93CF93DF93DC
:102D200080918A0182958F7009F069C08091870136
:102D3000882309F464C0A091BB01D091BC01B0917B
:102D40008501C0918601809188019091890121E0DF
:102D500030E0BF3F11F020E030E0122FBC01609561
:102D6000709506E04AC0009721F0CF3F29F4212F4B
:102D700005C021E030E002C020E030E020FD3BC093
:102D80004A2F50E0049FF001059FF00D1124E557F4
:102D9000FE4F2181C2132FC02081B2132CC022818B
:102DA000211129C0238134812817390718F0281BE5
:102DB000390B02C0260F371F283C3105E0F4809103
:102DC0008A018F70806180938A0186E0849FF00180
:102DD000859FF00D1124E057FE4F80818F70806138
:102DE000808385E891E00E944D12DF91CF911F9181
:102DF0000F910C945D16AF5FA770AD13B4CFDF9148
:102E0000CF911F910F910895EF92FF920F931F930F
:102E1000CF93DF93CDB7DEB762970FB6F894DEBFDE
:102E20000FBECDBF8C0185E0F801DE011D9601903B
:102E30000D928A95E1F7D8014C9111965C9111970A
:102E400012966C9112971396ED90FC9014977091D6
:102E50008501E09186018091880190918901009718
:102E600039F0EF3F41F421E030E07F3F31F003C023
:102E700021E030E002C020E030E020FD5CC1209184
:102E80008701222309F4F1C0E816F90628F097011A
:102E9000281B390BC90104C0809590958E0D9F1D8C
:102EA000883C910508F098C080918A01982F907F06
:102EB00009F064C0E51314C0741312C0611110C08E
:102EC0008F70806180938A010E947E1685E891E070
:102ED0000E944D1280918A01D80115968C9343C1AE
:102EE000EF2839F05F3F41F481E090E04F3F31F04F
:102EF00003C081E090E002C080E090E080FD03C06C
:102F000081E0862702C080E090E080FF2EC08091A3
:102F1000BB012091BC0136E013C090E0389FF00166
:102F2000399FF00D1124E557FE4F7181571306C0EC
:102F30007081471303C07281671317C001968770B1
:102F40008213EBCF12C19F7059F0882309F40BC193
:102F500007C09F7029F0F8019581907F09F403C1A3
:102F6000805E883008F4FFC0D2C0662309F4FBC03D
:102F700080918A01816080938A01F5C0E51308C0C1
:102F8000741306C0611104C0D80115968C939DC0BE
:102F90004D875E878D859E856A8B0E9419166A898A
:102FA000882309F4B4C0662309F4B1C020918A01D2
:102FB000822F82958F7090E002970CF4C6C08091AA
:102FC00085019091860198878F831986FB86EA8612
:102FD0002C87CE01079646C080918A01982F907F5A
:102FE00059F47E2DF98AE88A89890E943E1685E87F
:102FF00091E00E944D1295C0E51311C074130FC0EB
:1030000061110DC0F8018583C8010E944D12E5E8E9
:10301000F1E086E0DF011D928A95E9F7A2C04D87B5
:103020005E878D859E856A8B0E9419166A89882322
:1030300009F46DC0662309F46AC020918A01822FC9
:1030400082958F7090E002970CF47FC0809185018B
:10305000909186019A8389831B82FD82EC822E8364
:10306000CE0101960E944D1270C0E816F90628F0B4
:103070009701281B390BC90104C0809590958E0DCE
:103080009F1D883C910508F046C0662309F43FC0A7
:10309000E51330C074132EC020918A0120FD21C099
:1030A000322F32953F70832F90E00097D1F0D801F6
:1030B00015962C9315970F9741F0832F8F5F82956C
:1030C000807F2F70282B15962C93C8010E944D12DB
:1030D00086E0F801A5E8B1E001900D928A95E1F74C
:1030E0003EC086E0F801A5E8B1E001900D928A9516
:1030F000E1F737C04D875E878D859E850E94191642
:10310000811123C080918A01816080938A01C80166
:103110000E944D1226C07E2DF98AE88A89890E9474
:103120003E16E5E8F1E086E0DF011D928A95E9F7B9
:103130000E947E1618C0662351F34D875E878D85E9
:103140009E850E941916882311F386E0F801A5E8F0
:10315000B1E001900D928A95E1F70E948C160E94D1
:103160007E1681E014C080E012C04D875E878D8599
:103170009E850E94F81A292F22952F7030E0223068
:1031800031050CF4E0CE243031050CF6E2CE629627
:103190000FB6F894DEBF0FBECDBFDF91CF911F9168
:1031A0000F91FF90EF9008951F93CF93DF93CDB7CA
:1031B000DEB72C970FB6F894DEBF0FBECDBF4F839E
:1031C000588769877A878B879C87CE0107960E94EC
:1031D00004178823D9F02F8138858A859B85892B10
:1031E00039F03F3F19F080E090E004C02F3FD9F75D
:1031F00081E090E0892B09F06DC04F815885698589
:103200007A858B859C850E944D1664C086E0FE0100
:103210003796DE01119601900D928A95E1F7FF81B4
:10322000E8854A855B854115510539F0EF3F41F44A
:1032300081E090E0FF3F31F003C081E090E002C008
:1032400080E090E080FD46C02091BC0130E0C901E3
:103250000196877099276091BB0170E086179707E8
:1032600009F440C0F983EA835D834C8396E0929F22
:10327000D001939FB00D1124A557BE4FFE0131968A
:1032800001900D929A95E1F78093BC010E945D1622
:1032900021C0189FC001112485579E4F0E9404171A
:1032A000882371F1E091BB011E9FF0011124E557C5
:1032B000FE4F4081518162817381848195810E949A
:1032C0004D168091BB0190E00196877099278093FD
:1032D000BB0101C016E08091BB019091BC01891334
:1032E000D8CF0EC00E9415161092BC011092BB01DF
:1032F000E5E8F1E086E0DF011D928A95E9F7EACF83
:103300002C960FB6F894DEBF0FBECDBFDF91CF91E4
:103310001F910895DF92EF92FF920F931F93CF9327
:10332000DF93EC01009709F46EC0D12CEE24E394F6
:10333000F12C8E010F5F1F4FFE018491843748F4FA
:10334000843008F04CC0813071F0823009F05BC0ED
:103350001EC0853709F43FC080F1982F94589037EC
:1033600008F051C03FC02296F8018491982F905EDA
:10337000983050F48770FE2D01C0FF0F8A95EAF750
:103380008F2F0E948E1B13C00E9426112FC02296E1
:10339000F8018491982F905E983060F48770FE2D2C
:1033A00001C0FF0F8A95EAF78F2F0E94941B0E949D
:1033B000B71B1CC00E94EE1119C02296F80104919F
:1033C00007C08FE99FE00197F1F700C000000150AE
:1033D0000111F7CF0BC02296F801D49007C00E94CC
:1033E000261103C08F770E94EE11E8018D2D07C0D2
:1033F0008150EFE9FFE03197F1F700C0000088232A
:1034000009F497CFF5CFDF91CF911F910F91FF90E6
:10341000EF90DF9008956093C1017093C201809393
:10342000C3019093C4010C9403166093BD01709383
:10343000BE018093BF019093C0010C9403160895C0
:103440000C940B1A0F931F930091C1011091C201AC
:103450002091C3013091C401602B712B822B932BDF
:103460001F910F910C940B1A0F931F930091C101A0
:103470001091C2012091C3013091C40160237123D6
:10348000822393231F910F910C940B1A0F931F9378
:103490000091C1011091C2012091C3013091C4017A
:1034A00060277127822793271F910F910C940B1A85
:1034B00060E070E0CB010C94151A41E050E060E050
:1034C00070E004C0440F551F661F771F8A95D2F71E
:1034D000CB01BA010C94151A41E050E060E070E0B5
:1034E00004C0440F551F661F771F8A95D2F780913D
:1034F000BD019091BE01A091BF01B091C001482BC8
:10350000592B6A2B7B2BCB01BA010C94151A41E085
:1035100050E060E070E004C0440F551F661F771F45
:103520008A95D2F740955095609570958091BD0130
:103530009091BE01A091BF01B091C00148235923D1
:103540006A237B23CB01BA010C94151A41E050E0A9
:1035500060E070E004C0440F551F661F771F8A9516
:10356000D2F78091BD019091BE01A091BF01B091B1
:10357000C001482759276A277B27CB01BA010C9441
:10358000151A0F931F930091BD011091BE01209158
:10359000BF013091C001602B712B822B932B1F91A7
:1035A0000F910C94151A0F931F930091BD01109168
:1035B000BE012091BF013091C0016023712382239D
:1035C00093231F910F910C94151A0F931F93009141
:1035D000BD011091BE012091BF013091C001602753
:1035E0007127822793271F910F910C94151A089524
:1035F000CF92DF92EF92FF920F931F93CF93DF93BF
:10360000EC01C090C101D090C201E090C301F090E4
:10361000C4018091BD019091BE01A091BF01B09104
:10362000C001C82AD92AEA2AFB2A0FE110E0B70113
:10363000A601002E04C076956795579547950A9484
:10364000D2F740FF08C0BE01802F0E94FA038130EC
:10365000910509F007C00150110948F7BE0180E04B
:103660000E94FA03DF91CF911F910F91FF90EF908D
:10367000DF90CF90089540910C0150910D0120E012
:1036800030E09FEFFA01E20FF31F62816817A1F0AB
:103690009F3F19F4611101C0922F2F5F3F4F2630D9
:1036A000310581F707C0FA01E90FF11D97FDFA9581
:1036B000828308959F3FB9F7089540910C0150917E
:1036C0000D0120E030E0FA01E20FF31F9281981320
:1036D00001C012822F5F3F4F26303105A1F70895B8
:1036E00081E090E0E0910C01F0910D01E80FF91FED
:1036F0001082019688309105A9F708959091C5012F
:10370000982B9093C501089580959091C5019823B9
:103710009093C50108951092C50108959091C60136
:10372000982B9093C601089580959091C601982397
:103730009093C60108951092C60108958093C70121
:1037400008951092C701089540910C0150910D0108
:1037500020E030E080E0FA01E20FF31F9181911147
:103760008F5F2F5F3F4F27303105A9F70895E09114
:103770000C01F0910D018091C5018083E0910C0155
:10378000F0910D0180819091C601892B80839091E9
:10379000C701992361F0E0910C01F0910D01808146
:1037A000892B80830E94A41B81110E94A11B809100
:1037B0000C0190910D010C94F00F8091E701843081
:1037C00021F11092D10120E488E190E00FB6F89445
:1037D000A895809360000FBE2093600080E00E9457
:1037E000E10283B7817F846083BF83B7816083BF39
:1037F0007894889583B78E7F83BF88E10FB6F8945D
:1038000080936000109260000FBE0895089508959F
:10381000CF9380E00E94E1020E94061C0E943807BC
:103820000E94071CC0E08C2F0E948C08892B29F471
:10383000CF5FC530C1F780E001C081E0CF9108952E
:103840000E94151680E00E94E1020E94D0220E9490
:10385000E40F0C9462051F920F920FB60F92112481
:103860008F939F93AF93BF938091D101811113C028
:103870008091D2019091D301A091D401B091D50152
:103880004196A11DB11D8093D2019093D301A093C5
:10389000D401B093D501BF91AF919F918F910F90BB
:1038A0000FBE0F901F90189582E084BD93E095BDE8
:1038B0009AEF97BD80936E0008958FB7F89440916A
:1038C000D2015091D3016091D4017091D5018FBF85
:1038D000CA010895CF92DF92EF92FF920F931F9348
:1038E0002FB7F8944091D2015091D3016091D40147
:1038F0007091D5012FBF6A017B01EE24FF248C015A
:1039000020E030E0C016D106E206F30620F09A016E
:10391000281B390B05C09C0120953095240F351FBD
:10392000C9011F910F91FF90EF90DF90CF90089504
:103930001F920F920FB60F9211248F939F93AF9304
:10394000BF938091D2019091D301A091D401B09105
:10395000D5010196A11DB11D8093D2019093D30191
:10396000A093D401B093D501BF91AF919F918F9156
:103970000F900FBE0F901F9018950E94C80CF894DE
:103980002FEF87EA91E6215080409040E1F700C098
:10399000000087E090EBDC018093F1019093F2014D
:1039A000A093F301B093F4012CE088E190E00FB60E
:1039B000F894A895809360000FBE20936000FFCF1D
:1039C000CF92DF92EF92FF920F931F93CF93DF93EB
:1039D000C82ED12C01E010E08D2D0E948C087C01B6
:1039E000C0E0D0E098010C2E02C0220F331F0A94D1
:1039F000E2F72E213F21232B29F42196CC30D1054B
:103A000089F708C06C2F7D2D80E00E94D503C81275
:103A1000F4CF06C0D39485E0D812DECF80E001C099
:103A200081E0DF91CF911F910F91FF90EF90DF9098
:103A3000CF900895CF93C82F8CE20E94E01C88237A
:103A400021F08C2FCF910C94E01C80E0CF91089551
:103A5000CF930E946B1E811102C00E944C1EC5E6CE
:103A600008C00E9438078FE39CE90197F1F700C076
:103A70000000C150B1F789E20E941A1D81110AC1EC
:103A80008AE20E941A1D81110E944C1E85E00E944C
:103A90001A1D81110E94BD1C0E94761E8093D001C8
:103AA00087E00E941A1D882399F18BE10E941A1D5C
:103AB000882351F09091D00191FB882780F921E073
:103AC000822780FB91F922C08EE00E941A1D882374
:103AD00051F09091D00192FB882780F921E0822754
:103AE00080FB92F913C080E10E941A1D9091D001D1
:103AF000882341F093FB882780F921E0822780FB0F
:103B000093F904C0892F809580FB90F99093D001A0
:103B10008091D0010E947A1E0E94881E8093E1014C
:103B200080EE0E941A1D882341F08091E101982FB8
:103B3000909590FB80F98093E10189E30E941A1D22
:103B4000882359F09091E10191FB882780F921E0C9
:103B5000822780FB91F99093E10182EE0E941A1D69
:103B6000882359F09091E10192FB882780F921E0A8
:103B7000822780FB92F99093E10186EE0E941A1D44
:103B8000882359F09091E10193FB882780F921E087
:103B9000822780FB93F99093E10183EE0E941A1D26
:103BA000882359F09091E10194FB882780F921E066
:103BB000822780FB94F99093E10185E30E941A1D0E
:103BC000882359F09091E10195FB882780F921E045
:103BD000822780FB95F99093E10181E30E941A1DF1
:103BE000882359F09091E10196FB882780F921E024
:103BF000822780FB96F99093E10181E10E941A1DD2
:103C0000882359F09091E10197FB882780F921E002
:103C1000822780FB97F99093E1018091E1010E9456
:103C20008C1E87E20E941A1DC82F8EE10E941A1D69
:103C30008111C2608FE10E941A1D8111C46080E26F
:103C40000E941A1D8111C86081E20E941A1D811113
:103C5000C06182E20E941A1D8111C06283E20E944B
:103C60001A1D8111C06484E20E941A1D882311F07C
:103C7000C06802C0CC2329F08C2F0E94831E6C2FB9
:103C800003C00E947F1E682F70E080E090E0CF911B
:103C90000C94201ACF9108956DEE7EEF80E090E0B5
:103CA0000E94D92460E082E090E00E94CB2460E092
:103CB00083E090E00E94CB2460E084E090E00E94EA
:103CC000CB2460E085E090E00E94CB2460E086E0B9
:103CD00090E00C94CB2480E090E00E94C52421E089
:103CE0008D3E9E4F09F020E0822F089582E090E003
:103CF0000C94BD24682F82E090E00C94CB2483E0E8
:103D000090E00C94BD24682F83E090E00C94CB24C9
:103D100084E090E00C94BD24682F84E090E00C9443
:103D2000CB2486E090E00C94BD24682F86E090E0E0
:103D30000C94CB248091DE0180FF0BC060911101B7
:103D400085E0689FB0011124759567957595679515
:103D50002AC081FF09C06091110185E0689FB00110
:103D60001124759567951FC082FF07C060911101EE
:103D700085E0689FB001112416C04091D80144230A
:103D8000C9F060911001461788F72091110185E074
:103D9000289F90011124429FC001439F900D112440
:103DA00070E00E9495246038710540F4611571053A
:103DB00039F002C065E070E0862F08958FE708951E
:103DC00081E008958091DE0180FF08C060910F01BD
:103DD00070E0759567957595679521C081FF06C060
:103DE00060910F0170E07595679519C082FF04C05E
:103DF00060910F0170E010C08091D8018823C1F05C
:103E000060910E018617A0F790910F01989FC00155
:103E1000112470E00E9495246038710528F4611522
:103E2000710521F0862F08958FE7089581E00895A8
:103E300061E070E0F4CF803F21F40E949A1E8195EA
:103E400004C0813F29F40E949A1E8093DB010895EB
:103E5000823F21F40E949A1E819504C0833F29F479
:103E60000E949A1E8093DA010895893F19F40E94F6
:103E7000E21E05C08A3F31F40E94E21E81958093C4
:103E8000DC0108958B3F21F40E94E21E819504C05D
:103E90008C3F29F40E94E21E8093DD010895843F47
:103EA00021F48091D901816017C0853F21F4809170
:103EB000D901826011C0863F21F48091D9018460CC
:103EC0000BC0873F21F48091D901886005C0883FED
:103ED00031F48091D90180618093D90108958D3F9B
:103EE00021F48091DE0181600BC08E3F21F480912E
:103EF000DE01826005C08F3F29F48091DE0184607D
:103F00008093DE010895803F29F48091DB0187FFD3
:103F10006EC007C0813F41F48091DB0118160CF0A0
:103F200066C01092DB0163C09091DA01823F19F400
:103F300097FF5DC005C0833F31F419160CF057C0E0
:103F40001092DA0154C0893F31F48091DC011816D7
:103F50000CF04DC006C08A3F39F48091DC0187FF28
:103F600046C01092DC0143C08B3F29F48091DD01F3
:103F700087FF3DC006C08C3F39F48091DD011816E3
:103F8000B4F51092DD0133C0843F21F48091D90152
:103F90008E7F05C0853F31F48091D9018D7F80935C
:103FA000D90125C0863F21F48091D9018B7FF7CFBD
:103FB000873F21F48091D901877FF1CF883F21F499
:103FC0008091D9018F7EEBCF8D3F21F48091DE016E
:103FD0008E7F0BC08E3F21F48091DE018D7F05C066
:103FE0008F3F29F48091DE018B7F8093DE018091E9
:103FF000DA0181110EC08091DB0181110AC080912C
:10400000DC01811106C08091DD01811102C0109296
:10401000D801089589ED91E00E94FB0F0E945D1C7C
:104020009093D7018093D6010895CF938091D601C4
:104030009091D7010E946A1C4091D801442321F03D
:104040002091120130E006C0209113015AE0259F13
:10405000900111248217930708F486C08091DA0139
:1040600081110DC09091DB01911109C09091DC018B
:10407000911105C09091DD01992309F475C04F3F5E
:1040800019F04F5F4093D801181624F40E949A1E2D
:104090008093DA018091DA0187FF05C00E949A1EA1
:1040A00081958093DA018091DB01181624F40E9437
:1040B0009A1E8093DB018091DB0187FF05C00E947F
:1040C0009A1E81958093DB016091DA01662339F1B4
:1040D000C091DB01CC2319F1772767FD7095872FFD
:1040E000972F0E949A2323E333E343E35FE30E9485
:1040F000FE230E9467236093DA016C2F772767FD08
:104100007095872F972F0E949A2323E333E343E38D
:104110005FE30E94FE230E9467236093DB0180918E
:10412000DC01181624F40E94E21E8093DC018091C9
:10413000DC0187FF05C00E94E21E81958093DC01AF
:104140008091DD01181624F40E94E21E8093DD01A7
:104150008091DD0187FF05C00E94E21E819580935A
:10416000DD01CF910C940A20CF910895E9EDF1E0A3
:1041700085E0DF011D928A95E9F71092D80110922F
:10418000DE010895833089F130F4813061F08230AE
:1041900009F06EC019C0853009F449C0B8F1863005
:1041A00009F066C055C020911301862F90E0820F60
:1041B000911D8F3F910520F4620F609313010895C4
:1041C0008FEF80931301089520911201862F90E0C4
:1041D000820F911D8F3F910520F4620F60931201B1
:1041E00008958FEF80931201089520911101862F79
:1041F00090E0820F911D8F3F910520F4620F609334
:10420000110108958FEF80931101089520911001FD
:10421000862F90E0820F911D8F3F910520F4620F51
:104220006093100108958FEF8093100108952091FD
:104230000F01862F90E0820F911D8F3F910520F492
:10424000620F60930F0108958FEF80930F0108951F
:1042500020910E01862F90E0820F911D8F3F9105D6
:1042600020F4620F60930E0108958FEF80930E018A
:104270000895833021F130F4813059F0823009F013
:1042800049C012C0853089F128F1863009F042C05A
:1042900037C080911301681720F4861B80931301A7
:1042A000089510921301089580911201681720F467
:1042B000861B809312010895109212010895809137
:1042C0001101681720F4861B809311010895109244
:1042D0001101089580911001681720F4861B8093C6
:1042E0001001089510921001089580910F01681730
:1042F00020F4861B80930F01089510920F010895FA
:1043000080910E01681720F4861B80930E0108959A
:1043100010920E01089541E050E060E070E004C0AA
:10432000440F551F661F771F8A95D2F7CB01BA013C
:104330000E94201A0C941516873200F58E3108F071
:1043400086C08E3009F466C060F4873009F44DC031
:1043500018F4863049F531C0883041F18B3021F5B1
:104360007BC0863109F478C018F48031E9F45CC070
:10437000893109F471C08B31B9F442C0883309F432
:104380006BC048F4893209F460C0853309F45DC01C
:10439000873251F45AC0833409F457C018F48A3371
:1043A00018F057C0883499F080E008950E94761E76
:1043B0000E94881E0E94911E4FC08091D001817F73
:1043C0008E7F8093D00181E08093DF0108950E9469
:1043D00015162FEF83ED90E3215080409040E1F7D8
:1043E00000C000000E94BD1C37C08091D00180FF3A
:1043F00003C0817F8E7F01C081608093D0012CC07B
:104400009091D00191FB882780F921E0822780FBE1
:1044100091F913C09091D00192FB882780F921E097
:10442000822780FB92F909C09091D00193FB8827E5
:1044300080F921E0822780FB93F99093D0018823B3
:1044400059F091609093D00107C080E003C08D5176
:1044500001C089530E948B2181E0089580E0089576
:1044600080E00895CF93C82F8091DF01813071F0F3
:1044700020F0823009F089C037C0A0910C01B091C2
:104480000D018C91823209F082C007C0A0910C010D
:10449000B0910D018C91823249F48C2F0E942E2212
:1044A00081111EC08C2F0E949C211CC08C2F0E9449
:1044B0003022811115C0C43169F030F4CB3081F065
:1044C000C03109F068C009C0C93221F0C83309F011
:1044D00062C006C01092DF015EC082E08093DF01FF
:1044E00081E090E081705AC0C932C9F060F4C431F3
:1044F000B1F020F4C73009F04CC034C0CE51C63002
:1045000008F047C017C0CE3439F120F4CB3409F09D
:1045100040C01CC0C135C1F0C235D9F513C080916F
:10452000E001882319F01092E00133C081E080930C
:10453000DF0134C0EC2FF0E0E65BFE4F808180931A
:10454000E00127C061E003C061E007C06AE080913C
:10455000E0010E94C2201DC06AE08091E0010E943B
:10456000392117C08EE18093130182E380931201F9
:104570008AE08093110184E18093100188E08093A8
:104580000F0188E280930E0104C01092DF0180E0E9
:1045900005C081E003C080E090E0A4CFCF910895F2
:1045A0000E946B1E811102C00E944C1E0E94911E2F
:1045B0008093F00180FF02C0869501C080E00C94DA
:1045C000E1028091F001982F9695292F30E0233059
:1045D00031054CF49F5F990F8170892B8160809326
:1045E000F0010E94951E8091F00186950C94E102E5
:1045F0008091F001982F969591F09158990F8170C4
:10460000892B8093F0018E7F91E009F490E08091F6
:10461000F00190FB80F98093F0010E94951E80913B
:10462000F00186950C94E1028091F001982F90950D
:1046300090FB80F98093F0010E94951E8091F0011B
:1046400080FF02C0869501C080E00C94E1023091A9
:10465000F001232F26952F5F2F77822F90E0317066
:1046600004972CF4220F232B2093F00102C03093E7
:10467000F0018091F001282F2E7F91E009F490E065
:1046800090FB80F98093F0010E94951E8091F001CB
:1046900086950C94E1022091F001922F969598272F
:1046A000990F822F8170892B8093F0018E7F91E08A
:1046B00009F490E08091F00190FB80F98093F00183
:1046C0000E94951E8091F00186950C94E10204D021
:1046D0006894B1118DC0089570D088F09F5790F004
:1046E000B92F9927B751A0F0D1F0660F771F881F17
:1046F000991F1AF0BA95C9F712C0B13081F077D07E
:10470000B1E0089574C0672F782F8827B85F39F01B
:10471000B93FCCF3869577956795B395D9F73EF475
:1047200090958095709561957F4F8F4F9F4F08951D
:10473000E89409C097FB3EF490958095709561953B
:104740007F4F8F4F9F4F9923A9F0F92F96E9BB27F1
:104750009395F695879577956795B795F111F8CF6D
:10476000FAF4BB0F11F460FF1BC06F5F7F4F8F4FD8
:104770009F4F16C0882311F096E911C0772321F0CE
:104780009EE8872F762F05C0662371F096E8862F66
:1047900070E060E02AF09A95660F771F881FDAF7BD
:1047A000880F9695879597F9089557FD9058440F6F
:1047B000551F59F05F3F71F04795880F97FB991F80
:1047C00061F09F3F79F0879508951216130614063D
:1047D000551FF2CF4695F1DF08C0161617061806CA
:1047E000991FF1CF86957105610508940895E894A5
:1047F000BB2766277727CB0197F908950BD078C0A0
:1048000069D028F06ED018F0952309F05AC05FC027
:104810001124EECFCADFA0F3959FD1F3950F50E09E
:10482000551F629FF001729FBB27F00DB11D639F62
:10483000AA27F00DB11DAA1F649F6627B00DA11D08
:10484000661F829F2227B00DA11D621F739FB00DAE
:10485000A11D621F839FA00D611D221F749F33271E
:10486000A00D611D231F849F600D211D822F762FB7
:104870006A2F11249F5750408AF0E1F088234AF0B4
:10488000EE0FFF1FBB1F661F771F881F9150504000
:10489000A9F79E3F510570F014C0AACF5F3FECF31B
:1048A000983EDCF3869577956795B795F795E795EC
:1048B0009F5FC1F7FE2B880F911D9695879597F9FD
:1048C000089597F99F6780E870E060E008959FEF92
:1048D00080EC089500240A94161617061806090697
:1048E000089500240A941216130614060506089566
:1048F000092E0394000C11F4882352F0BB0F40F4EE
:10490000BF2B11F460FF04C06F5F7F4F8F4F9F4F2D
:104910000895991B79E004C0991F961708F0961B1B
:10492000881F7A95C9F78095089597FB072E16F48E
:10493000009407D077FD09D00E94A92407FC05D078
:104940003EF4909581959F4F0895709561957F4FA6
:104950000895AA1BBB1B51E107C0AA1FBB1FA617C6
:10496000B70710F0A61BB70B881F991F5A95A9F718
:1049700080959095BC01CD010895F999FECF92BD27
:1049800081BDF89A992780B50895A8E1B0E042E08A
:1049900050E00C94E024262FF999FECF1FBA92BD67
:1049A00081BD20BD0FB6F894FA9AF99A0FBE019610
:1049B00008950E94CB24272F0C94CC24DC01CB013A
:1049C000FC01F999FECF06C0F2BDE1BDF89A31961F
:1049D00000B40D9241505040B8F70895F894FFCFBD
:1049E00005960826090209CD08990801C80128087A
:1049F000140A321E420045002500260043006100D3
:104A00006000200037006400650066006700440015
:104A100046002400470074038D03A603BF038B04E4
:104A20003E040804E8033F4D362001020304050656
:044A3000070809006A
:00000001FF
